:10000000220B130A530A670A070A260A730A040016
:1000100045060E0A61006505C304120AE107120ACB
:100020006504C30500084507200AC306250A4507DD
:100030001F0A0400E1071E0A6504250A170A250A9B
:100040004506250A04006100200A0008010C36005C
:100050001402960043062E0A0306440A13095B0C99
:100060002800E802310A000000002506390A0304CE
:100070003A0A0305350313095B0C2800E8023E0A1F
:1000800000000000B602280A080C280014028800AC
:10009000290029024306500A03043503E9024C0AE9
:1000A00015022900000819024306660A010C2900FE
:1000B000BF0C28000400E8025A0AE902580A2E0C74
:1000C0002800E802610A0400F902560A0008FC0C44
:1000D0007A013A033A031A024306720A700A0400CC
:1000E000FA02700A0008C306210B010C3700150242
:1000F000970043067D0A0306210B1309030434030A
:100100000306840A1804850A18051806890A0504D6
:100110008A0A0505010C390053090504A3079C0A46
:10012000010C39005309040C3900B30C3A0067097B
:10013000F902950A0000A60A020C39005309070CBF
:100140003900210C3A006709F902A10A1806AA0A27
:100150000504AB0A0505010C390053090504A30782
:10016000BD0A010C39005309040C3900B30C3A00E4
:100170006709F902B60A0000C70A020C39005309E0
:10018000070C3900210C3A006709F902C20A180667
:10019000CB0A0504CC0A0505010C390053090504F6
:1001A000360243071F0B13091807D80A0504D90A9A
:1001B0000505010C390053090504A307EB0A010CDE
:1001C00039005309040C3900B30C3A006709F902ED
:1001D000E40A0000F50A020C39005309070C390043
:1001E000210C3A006709F902F00A1807F90A050418
:1001F000FA0A0505010C390053090504A3070C0B85
:10020000010C39005309040C3900B30C3A0067099A
:10021000F902050B0000160B020C39005309070CFC
:100220003900210C3A006709F902110B18071A0B63
:1002300005041B0B0505010C390053090504B70221
:10024000770A0008180C2700080C2400000C200076
:10025000A402E702270B6400F60C05007F0C0600E1
:100260000504E6046505050C02004507390B04008A
:10027000350B45063D0B0400390B61004507420B69
:1002800004003E0B01022F00A10C8F0003064B0B54
:100290006F0C8F000307390B830C8F000306520B82
:1002A000A305530BA304060C0200610007092507F0
:1002B0005B0BA607560BA607900B2507900BC607EE
:1002C0007F0B06021F0E2F00E60513052F024307C2
:1002D0006B0BB202780B1F0C8F004307770B030CDC
:1002E00092000307770B720070007100900B720090
:1002F0000A0CD00124000F022000B002900B0D0C5C
:10030000D101240000022600600C06001305E6055A
:10031000310243078F0B0F0C6D01B102900B71007E
:100320002506A00B020C34002609040C3400260913
:100330000902100D2D00050C3400260909022E00BB
:100340001307AA0BA607A80B07092507900BA20BFA
:10035000E60413047F0C0600030C90004307E40B33
:10036000100C8A000306E30B200C8B000306E30B42
:100370002C024306E30B0400070C3400040C350088
:10038000010C360073090A023400040C35007600B3
:1003900073090B023400050C3500760073090C025A
:1003A000EC00120C8B004306D90B1A0C8B00430790
:1003B000DC0B2C024307E20B7400060C3500010C29
:0C03C00036007309B80B7000560B0300E8
:0203FE00000AF3
:021FFE00FD0FD5
:080400000000010000000000F3
:00000001FF
